:10000000830100308A002F28A00003088301B1007B
:100010000B1D0B280C281728A108031910281128DC
:100020001328043085068312210A81000B118312E4
:100030000C1C1B281C282928A20803192028212869
:100040002328023085068312220A8E00FF308F009B
:100050000C10831231088300A00E200E09002130FD
:1000600084002C30412083010330B000FE30AF000B
:100070002C3084002D3045208301AA2904068001FC
:10008000840A0406031D3E280034AD005020800081
:10009000840A04082D060319003446288312AF0091
:1000A000B01B592830088A002F08AF0A0319B00A7C
:1000B00082008313301883172F08AF0A84000008CA
:0200C000080036
:1002EA00A701A801AB009A2983122C08AD00AE0120
:1002FA000310AD0DAE0D0310AD0DAE0D0310AD0D17
:10030A00AE0D2D08A9002E08AA008B29FF308312F2
:10031A00A907031CAA032A082904031D952996295B
:10032A008B298312A70A0319A80A83122B08AD0086
:10033A00AE0128082E06031DA42927082D06031D31
:10034A00A729A829792983120800A301A401073043
:10035A00990083169F01FF30850083128501FF30C3
:10036A008F008E01A101A2013130900082308316E4
:10037A0081000B17831281018B1683160C148B17BD
:10038A00643083127521F930831685008312850142
:10039A00FC2B78308312AC005030A100BC30A20094
:1003AA001830831275217530A100183075218C30F0
:1003BA00A10018307521AA30A10018307521143017
:1003CA00A100B330A200183075214530A1001830C1
:1003DA0075216430A100183075218C30A1001830C5
:1003EA0075212E30A100AA30A20018307521503094
:0603FA00A100183075217E
:100400007530A100183075219930A1001830752180
:100410007530A100A430A200183075211430A1005D
:10042000183075214530A100183075217530A100B4
:10043000183075217D30A1009930A2001830752147
:100440002E30A100183075215030A10018307521D0
:100450007D30A100183075215030A1008C30A200F1
:10046000183075217530A100183075211430A100A5
:10047000183075215030A100183075217D30A10051
:100480009930A200183075215030A1001830752124
:100490006430A100183075212E30A100183075216C
:1004A0001430A100A430A200183075214530A100FD
:1004B000183075216430A100183075218C30A100EE
:1004C000183075215030A100D630A20018307521A7
:1004D0007530A100183075218C30A100BC30A2000D
:1004E00018307521AA30A100183075211430A100F0
:1004F000C730A200183075214530A1001830752191
:100500006430A100C030A200183075218C30A100E9
:10051000183075212E30A100BC30A2001830752192
:100520005030A100183075217530A100AA30A2000A
:10053000183075219930A100183075217530A1004F
:10054000BC30A200183075211430A100183075217C
:100550004530A100B330A200183075217530A100DC
:10056000183075217D30A100AA30A2001830752105
:100570002E30A100183075215030A1009930A20012
:10058000183075217D30A100183075215030A10040
:10059000AA30A200183075217530A10018307521DD
:1005A0001430A100C730A200183075215030A100CE
:1005B000183075217D30A100C030A200183075219F
:1005C0005030A100183075216430A100CE30A20057
:1005D000183075212E30A100183075211430A1007B
:1005E000D630A200183075214530A1001830752191
:1005F0006430A100183075218C30A100D430A200E5
:10060000183075215030A100AA30A2001830752191
:10061000A430A200183075217530A100AA30A200C4
:10062000183075215030A200183075211430A10007
:10063000A430A200183075218C30A200183075212A
:100640007D30A1006430A200183075217530A20001
:10065000183075212E30A1005030A20018307521BD
:10066000AA30A200183075215030A100A430A20099
:10067000183075219930A200183075217530A1000D
:10068000A430A20018307521BC30A20018307521AA
:100690006430A100C730A20018307521CE30A2000E
:1006A000183075215030A100C030A20018307521DB
:1006B000BC30A200183075212E30A100B330A2004A
:1006C00018307521C030A200183075215030A100BB
:1006D000BC30A20018307521B330A200183075214B
:1006E0007530A100AA30A20018307521A430A200F4
:1006F000183075216430A1009930A200183075219E
:100700008C30A200183075215030A1007D30A2003D
:10071000183075219930A200183075214530A1009C
:100720008C30A200183075219930A2001830752144
:100730006430A1008C30A200183075217D30A200F9
:10074000183075215030A100AA30A2003030752138
:100750007530A100BC30A200303075218C30A10072
:10076000B330A200303075217D30A10030307521CA
:100770007530A100303075212E30A100AA30A200C2
:10078000303075215030A100BC30A20030307521CE
:100790006430A100303075215030A100CE30A2006D
:1007A000303075212E30A100303075212E30A1005F
:1007B000C730A200303075217530A100303075216E
:1007C0006430A100AA30A200303075215030A10061
:1007D000C030A200303075214530A100B330A200F6
:1007E000303075216430A100C730A200303075214F
:0E07F000A101A20118307521CE292F28B034A6
:02400E0004317B
:00000001FF
